:020000020000FC
:0200000014C02A
:0200160028C000
:1000260069C045C00FED0DBF00E007BB0FEF08BB71
:1000360000E001BB0FE702BB02E00ABB01E00BBB1D
:1000460008E30BBF0FE705B901E004B90FEF00BDE8
:1000560000E305BF00E808B90FE006B97894889573
:10006600FECF16B31F3789F01F3B89F01F3D89F07D
:100076001F3E89F0173F89F01B3F89F01D3F89F02D
:100086001E3F89F001E00BBB189517E00EC016E085
:100096000CC015E00AC014E008C013E006C012E068
:1000A60004C011E002C010E000C02FD0DACF10B3B8
:1000B6001F771F3379F01F3579F01F3679F0173720
:1000C60079F01B3779F01D3779F01E3779F001E0AA
:1000D6000BBB18951EE00CC01DE00AC01CE008C052
:1000E6001BE006C01AE004C019E002C018E000C018
:1000F6000CD0DDCF19B31170103019F001E00BBB35
:1001060018951FE000C001D0F5CF24E03DD013FFC5
:100116002DD013FD32D038D012FF28D012FD2DD0AD
:1001260033D011FF23D011FD28D02ED010FF1ED0C2
:1001360010FD23D029D013FD19D013FF1ED024D0D3
:1001460012FD14D012FF19D01FD011FD0FD011FFD0
:1001560014D01AD010FD0AD010FF0FD015D00DD034
:100166000CD00BD00AD02A9589F6089530E148E0E4
:100176004A95F1F73A95D9F7089530E448E04A955B
:10018600F1F73A95D9F7089530E103E00BBB00008B
:1001960042E04A95F1F701E00BBB000044E04A95C6
:0801A600F1F73A9591F7089575
:00000001FF
